:1000000000308A0000290000AB0CAA0CAB0CAA0C33
:100010003F30AB05A90CA80CA90CA80CA905AB088E
:10002000031D16282A087F3C031827283030A1001A
:1000300080302A02B3002B08B4000030031C0130CA
:10004000B4020310330DAC00340DAD00362831304E
:10005000A1002A087F3CB300B4012B08031C2B0F1E
:10006000B4020310330DAC00340DAD00A908031D1C
:100070003D2828087F3C03186A288030A8020030F9
:10008000031C0130A9022D082902031C5028031D5E
:100090004D2828082C0203185028B101B001592816
:1000A00028082C02B0002D08B1002908031C290FD4
:1000B000B10228082C07AE002D08AF00290803184C
:1000C000290FAF072F08003C03186928AF01FF3044
:1000D000AE009B2828087F3CA8002908031C290F94
:1000E000732800307428003CA9002D082902031C45
:1000F0008228031D7F2828082C0203188228AF01BC
:10010000AE018B2828082C02AE002D08AF0029086C
:10011000031C290FAF0228082C07B0002D08B100DE
:1001200029080318290FB1073108003C03189B2840
:10013000B101FF30B0008A110A126B292108A20018
:100140002F0CB5002E0CB400B50CB40CB50CB40CCF
:10015000B50CB40C0F30B50530303407A3002E08B1
:100160000F39B400B50130303407A4002108A500D0
:10017000310CB500300CB400B50CB40CB50CB40C9B
:10018000B50CB40C0F30B50530303407A60030087C
:100190000F39B400B50130303407A70053300C1EBE
:1001A000CF28990053300C1ED3289900B30133088F
:1001B000053C031CE7282230330784008313000822
:1001C000B40034080C1EE2289900B30AD728B30102
:1001D0003308053C031CF9282230330784008313BD
:1001E0000008FF3AB40034080C1EF4289900B30A42
:1001F000E82845300C1EFA2899008A110A126C2949
:10020000840183131F308305403083169900A23088
:10021000980090308312980083161F149F141F15A6
:100220009F1107309C008312A001FF30B200803084
:10023000831687008312B200F030831686000B30DD
:1002400085008113831232103208831687008312CF
:10025000071083161F109F101F159F111F13831265
:100260001F139F1783169F1783121F14B210320893
:100270008316870002308312870683160511043027
:10028000831285060030F8001F08C73978049F00E4
:100290001030F700F70B4A2900001F151F194E29CF
:1002A00083161E088312AA001E08AB000830F8004F
:1002B0001F08C73978049F001030F700F70B5E293C
:1002C00000001F151F19622983161E088312A8003B
:0C02D0001E08A90004289E28362963009F
:02400E00723FFF
:00000001FF
